:020000040000FA
:100000000E22532197212B28AD0A0B11090005342C
:1000100008343D3412340434823407340E3404344A
:10002000813403341034B23466346034B1348F34E4
:1000300043345034003420344F346834363461341F
:10004000633420344C34433420346D346534743498
:10005000653472340034F7208514061BA028C901CA
:10006000C90A061F44200230D320A9210D306D217A
:10007000363049183A306D211730E0210310B32390
:100080003521073018223128C90AC91085144918AA
:1000900085106121061B0800C901A9215C212F30B0
:1000A0006D215821CB007421CA004907940014081F
:1000B000203003195E282B30941B2D307A21941F99
:1000C00063289409940AAB2235213B0E0F39303E48
:1000D0007A216F223B080F39303E7A2125307A2170
:1000E00072222A30C90803197A2161215321031D84
:1000F0008828061B4D284A084907323C03198228E4
:10010000C90A4D28CE304A02FF3A013EC9004D28A7
:10011000490803199F28CA074A0888004B08890024
:10012000831688189128081555308900AA3089004F
:10013000881483122A307A216121A92161214C2857
:10014000A92164211B30C30090226121A9215C21D7
:1001500025306D21CA200319A0283630E0218510F2
:100160006121CA200319A0283230E02185146121C1
:10017000A921B521AB215C2116306D21CA200319BC
:10018000C228FB281A306D21B9281F30C328FC3043
:100190002D050800CC0BCD2886165321031D002801
:1001A000061F002804300B11AE01AD018101C30010
:1001B0008B168B1783160514831205146421C30B49
:1001C000DE2883160510831205108B130108AC007E
:1001D000AB018316011601128312AB0301082C0632
:1001E0000319E9282D082C042E308C0008008612F3
:1001F0002830CC000800BD21BB21A301861F0C299B
:10020000CA21FE21CC2117210B30C3000F3023055A
:10021000031DC5281922B928CC21F021CC210222A6
:10022000D121CC21D721CA2117210F300529BF01A7
:10023000BE01E830BC000330BD0058217421801B92
:100240002529BC070318BD0A2629BC070022CC219A
:10025000E830BC000330BD000022D721CA21203085
:10026000971B2D307A219713AF222030A400B701BD
:10027000B801B901BA01BB01373084000530A600CE
:10028000333080078019F039801B0F398002840ACF
:10029000A60B4029AE23BB0DBA0DB90DB80DB70D95
:1002A000A40B3C29080080300605A902A90008001B
:1002B0000130861F0030080072224330861F4C3008
:1002C0007A296221642164217E30A7001230A800BF
:1002D000A80F6829A70F6829003489007521031920
:1002E00008007A21890A6E2989008316081483126E
:1002F00008080800C20AC00B8429C100061A832915
:10030000C030B921922141088515AA002A0E892101
:100310002A080F39A500F030860525088604051542
:10032000000005114230A700A70B94290034642176
:10033000851105110330892164210330892103309F
:100340008921023089210C30812128308121063019
:100350008121013081210930C0000230B921C20160
:10036000FD30A7006630A8006829421A08007222F2
:10037000B529851185290622BF293230072202229C
:10038000CA21D121CC21D121AB227F309800D721A5
:100390006523CD290623CD29D02221308C001D30A4
:1003A000E0291D308C002130E0211830CE291D308D
:1003B0008C001130E0211830CE2111308C00183023
:1003C0008D000430A6000C0884000008C4000D084D
:1003D0008400440880008C038D03A60BE3290800E9
:1003E0001330C300D12118308400C70147158E2275
:1003F0008000C30A8403C70BF72908001730F129CE
:100400003F30072A3630072A3230072A2E30A40020
:10041000D12124088C001730E021972A8316273039
:10042000810010308500D0308600831285010800DD
:10043000C300F221971F1D2A97130A30C500C70178
:100440001808C60074220319282A303E7A21542A3B
:100450004718522A45030319522A45089D00C5032F
:1004600074220319452A180AC502031C452AC50A25
:100470007422043C0318452AC50A742280220319F9
:100480003C2A1D0845020319222A1D08C500170B26
:100490004D2A04304502031C522A45084602031C1B
:1004A0005A2A592A30307A214714980303196A2AA4
:1004B0005A2A7222C50303196A2AC718692A970B98
:1004C000692A47186F22C718692A03309700960ACD
:1004D000960A222A722216086D2115086D29C71462
:1004E0002E307A2920307A294508013E8400040CF8
:1004F0003C3C84000008451C000E9B000F3908009E
:100500007422013ECA000A3C0319CA011B08F039D3
:100510004A048000451C800ECA0808004308820077
:100520008E22003E031908007A21C30A902A9E30C9
:100530009800A201971F9F2AB823C622A217031072
:10054000971BA62AAE23980BA02A612BA21F9713F4
:1005500000349401980197019601950100349401AB
:100560001808031900341708A20097179E30980244
:10057000981FCE2A9809980A18080319C32A03104D
:10058000B323980BBF2AA21F0034B823940A03197F
:10059000950A0319960A0319970A00342314FF34A5
:1005A0001808031D1D080319A92A17081C06A20014
:1005B0001D0898077E30031CE12A98020318042BBB
:1005C000E42A9802031C612BBD2394179C17031087
:1005D000AB221830A500121CF72A1A0895071B0831
:1005E00003181B0F96071C0803181C0F9707B3234B
:1005F000930C920C0310A50BEB2A971B012BAE2337
:100600009803A21F97130034A314FF341D08031985
:10061000632B18080319A92A17081C06A2009717AC
:100620009C17A501BD231A0892021B08031C1B0F6F
:1006300093021C08031C1C0F940294019301920165
:10064000031C262B0310B3230130A5001D089802BC
:10065000031C302B7E30250798070318042B352BFD
:100660007E3025079807031C612B1830A400920DDB
:10067000930DAE23A50D1A0895021B08031C1B0F32
:1006800096021C08031C1C0F97021C0DA504251CB8
:100690004B2B1214562B1A0895071B0803181B0F17
:1006A00096071C0803181C0A97071210A40B372B77
:1006B000A21F9413140897001308960012089500BF
:1006C00000342315FF34A315FF3480309C0617082F
:1006D0001C06A5009401990118081D020318D721D2
:1006E0001D08031900341708A20097179C171D084E
:1006F00018029D000319832B03109C0C9B0C9A0C71
:10070000990C9D0B7C2BA51F902B99099A099B098D
:100710009C09990A03199A0A03199B0A03199C0A4E
:10072000190894071A0803181A0F95071B080318CD
:100730001B0F96071C0803181C0F9707A51BA62B59
:10074000031CA62AB323980FA62A042B03189F2A5A
:10075000B823C6228030A20694019F2A940D950DDD
:10076000960D970D0800970C960C950C940C0800AC
:100770009409950996099709080017089400160826
:08078000930015089200080027
:02400E00F23F7F
:10420000000000002500200000006D000000750087
:1042100000006E000000700000002000460000005A
:10422000480000006B0048007A00000020003D00BC
:10423000200000003F003F003F003F0000002A0038
:104240006D00610078002A0000003A0020007A002A
:10425000650072006F0069006E00670000002000BA
:10426000610064006A003A002000000031003A005A
:0C4270002000000032003A002000000096
:00000001FF
